:020000040000FA
:060000000A128A11A62875
:08000800FF00030E8301C0009C
:100010000A08C1008A017E08C4004208C30004081F
:10002000C8002008B0002108B1002208B20023084F
:10003000B3002408B4002508B5002608B600270838
:10004000B7002808B8002908B9002A08BA002B0808
:10005000BB002C08BC002D08BD002E08BE002F08D8
:10006000BF008A11862F820740343034183411348F
:10007000153420342030C2000310A80DA90DAA0D9C
:10008000AB0D0310A00DA10DA20DA30D031C56284E
:100090002408A80725080318250FA9072608031810
:1000A000260FAA0727080318270FAB07C20B3C2807
:1000B00008002030C200A401A501A601A701031079
:1000C000AC0DAD0DAE0DAF0D0310A00DA10DA20D29
:1000D000A30DA40DA50DA60DA70D27082B02031D2A
:1000E0007B2826082A02031D7B2825082902031DD8
:1000F0007B282408280203197F2803188E28280843
:10010000A4022908031C290FA5022A08031C2A0F90
:10011000A6022B08031C2B0FA7022C14C20B5F286E
:100120000800C71BA228471B9D284608840083138C
:10013000C708031D8317000808004608C5004708C4
:100140003F39A32808008A0046088200831606105B
:1001500086100611861106168616061786170511D3
:100160008511051205138513CE2983160313AC15CB
:100170002C088312850083162C122C08831285000C
:100180000317A601A31BC828831603132C11CB2821
:10019000831603132C152C08831285008316AC11CB
:1001A0002C088312850003100317A20DA30D8312E0
:1001B00003130530A0000A128A11A00BDD28831654
:1001C000AC152C08831285000317A60A10302602EE
:1001D000031DC228831603132C162C0883128500D6
:1001E0000800D8004E088312A00083164F0883121F
:1001F000A100831650088312A200831651088312AF
:10020000A3000530A400A501A601A7013A2083128E
:10021000031328088316DA00831229088316DB00EB
:1002200083122A088316DC0083122B088316DD0054
:10023000EC01EC014E08E400E501E601E701640889
:100240008312A000831665088312A1008316660836
:100250008312A200831667088312A300B830A4009B
:100260006330A5005E30A600A7018A113A208312F0
:10027000031328088316E400831229088316E50077
:1002800083122A088316E60083122B088316E700E0
:100290006C088A11031D51296708E400E501E60195
:1002A000E70101306C02031D5B296608E400670862
:1002B000E500E601E70102306C02031D66296508CE
:1002C000E4006608E5006708E600E7016408DA076D
:1002D00065080318650FDB0766080318660FDC075F
:1002E00067080318670FDD074F08CE005008CF00DE
:1002F0005108D000D101EC0A04306C02031D1A2908
:100300005A0883120317A0003F30831603135B05BE
:1003100083120317A100831603135808031D9429A1
:10032000831203172117972983120317A117200897
:10033000A2002108A300B520831603135B08DA008E
:100340005C08DB005D08DC00DD0106308312A000E4
:1003500003108316DC0CDB0CDA0C83128A11A00B61
:10036000A82983165A0883120317A0003F3083166A
:1003700003135B0583120317A100831603135808A8
:10038000031DC629831203172117C92983120317D6
:10039000A1172008A2002108A300B5281430831259
:1003A000E800E030E900B830EA001530EB008A15CB
:1003B0006429A70028080319E42983160313AD153F
:1003C0002D0883128600EA2983160313AD112D0828
:1003D0008312860003172708AB00A901342A2508D9
:1003E0000313C7000317290824070313C6000318C3
:1003F000C70A912083120317AA002E302A028A11FD
:100400000319332AAD01831603132D102D0883120F
:100410008600803003172A05AC002C080319172A20
:1004200083160313AD142D08831286001D2A83162C
:100430000313AD102D088312860083162D142D088A
:100440008312860003100317AA0D831203130530CD
:10045000A0000A128A11A00B2B2A0317AD0A08303C
:100460002D02031D032AA90A29082B02031DEF29C7
:10047000080083162D112D088312860083120313A2
:100480005F30A0000330A1000A128A11A10B442A98
:100490000A128A11A00B422A000000003430031710
:1004A000A40000304038A5000130A8000630D92152
:1004B000831603132D152D08831286000800803043
:1004C00083160313EC009630ED009830EE00EF0138
:1004D000E2015E086207840083135F1883170F3000
:1004E0008000E20A0C306202031D692A0730E40032
:1004F00083120317A401831603136C088312A80048
:1005000083166D088312A90083166E088312AA0051
:1005100083166F088312AB0083164E088312A00067
:1005200083164F088312A100831650088312A2007D
:10053000831651088312A3005920831203132C0839
:100540008316E8006808831203172715031927117B
:1005500083160313640A83120317A600831603137A
:100560005E08831203172607840083138316031380
:100570005F1883170F30000283120317A711031DA2
:10058000A7152712271DA71927168A11271ED22A59
:10059000831603135E086407840083135F188317B0
:1005A000680880008312031324088316CE00831288
:1005B00025088316CF00831226088316D0008312E5
:1005C00027088316D1000A308312A800A901AA01C6
:1005D000AB0183166C088312A00083166D0883128A
:1005E000A10083166E088312A20083166F0883127F
:1005F000A3005920831203132C088316EC008312E6
:100600002D088316ED0083122E088316EE00831248
:100610002F088316EF00E40383120317A40A0730A0
:1006200024028A11031D7B2A831603135E088400AB
:1006300083135F1883174E08800083120317271C4B
:10064000972B831603135908803A8312A000803039
:100650002002031D2E2B0030831658020319432B52
:100660000318432B83165E080B3E840083135F1828
:1006700083170A3080005809E9005909EA00E90A9D
:100680000319EA0A482B83165808E9005908EA00BA
:1006900064308312A800A901AA01AB01831669087E
:1006A0008312A00083166A088312A100A201A3018D
:1006B0005920831603135E080A3E840083135F18D3
:1006C000831783122C08800024088316E900831204
:1006D00025088316EA000A308312A800A901AA019E
:1006E000AB01831669088312A00083166A0883127F
:1006F000A100A201A3018A115920831603135E08E9
:10070000093E840083135F18831783122C0880002E
:1007100024088316E900831225088316EA005E0880
:10072000083E840083135F1883176908800008005F
:10073000D8001530DA002030DE00EB012D112D0835
:1007400083128600831203135F30A0000330A100E0
:100750000A128A11A10BA82B0A128A11A00BA62B30
:1007600000000000DE300317A400A5010130A8003E
:100770000130D921DA3083120317A400A50101301A
:10078000A80001308A11D921831603134E08E8000E
:100790006808EC00E4018A11D82B5408640784002F
:1007A0008313551883172E300002031DEB0AE40A49
:1007B00064086C02031DCD2B6B08580783120317C6
:1007C000A000200983160313E9000D30E9076B0828
:1007D000580783120317A0002008031DF42B0B30C9
:1007E00083160313E900042C831603136B085807C0
:1007F00083120317A0000C3020020319042C031CE1
:10080000042C83160313E901031083160313690DE7
:1008100083120317A000E030200483160313E000C6
:10082000E03083120317A400A5010130A8000130B5
:10083000D92183160313540883120317A4008316C7
:100840000313550883120317A500A8010D308A1160
:10085000D92183160313E401540864078400831329
:10086000551883172E300002831203172212031922
:100870002216831603136408580283120317A21268
:10088000031D031CA2162217221AA21E22138A116C
:10089000221F602C83160313580864028312031767
:1008A000A0000310200DA100E03021070313E90090
:1008B00068300317A400A5010130A8000430D92135
:1008C00083160313E40A0D3064028A11031D2C2CD5
:1008D0002D152D088312860008008316CE000C30DB
:1008E0004E020319772C031C772C0C30CE002D11EF
:1008F0002D0883128600831203135F30A00003309B
:10090000A1000A128A11A10B812C0A128A11A00BD4
:100910007F2C0000000083164E09D2000D30D20754
:100920000C3052020319982C031C982C0C30D20066
:100930000310520DD400E03054048312E9006830F3
:100940000317A400A5010130A8000430D9218316A3
:1009500003132D152D088312860008005A08E200A3
:100960005B08E3009C1CB52CB22C62089B001C1495
:100970001A08E000600808008316E0005A08E40046
:100980005B08E5009C1CC52CC22C64089B00600819
:100990009A001C1562108B1B62148B1355309D003E
:1009A000AA309D009C146218D72C8B13D82C8B175F
:1009B0001C1108004C08D6004D08D7005608DA0074
:1009C0005708DB00AE2483160313D20001304C0716
:1009D000D6000030031801304D07D7005608DA0062
:1009E0005708DB008A11AE2483160313D3000800D6
:1009F0004C08D6004D08D7005608DA005708DB002F
:100A00005208BC240130831603134C07D600003073
:100A1000031801304D07D7005608DA005708DB00ED
:100A200053088A11BC2CE8305A02A00003305B0244
:100A30002004031D1E2D0930C900080064305A022D
:100A4000A00000305B022004031D292D0A30C900DC
:100A500008000A305A02A00000305B022004031D87
:100A6000342D0B30C900080001305A02A0000030BC
:100A70005B022004031D3E2D0C30C90008006C08E9
:100A8000DC006D08DD0001306C02A00000306D025A
:100A90002004031D4F2D0A30DA00DB01132D0A302C
:100AA0006C02A00000306D022004031D5B2D643039
:100AB000DA00DB01132D64306C02A00000306D02FF
:100AC0002004031D672DE830DA000330DB00132D0E
:100AD0006E08DC006F08DD00E8306E02A000033015
:100AE0006F022004031D782D6430DA00DB01132D22
:100AF00064306E02A00000306F022004031D842DBC
:100B00000A30DA00DB01132D0A306E02A00000303B
:100B10006F022004031D8F2D0130DA00DB01132D3D
:100B200083125C085A02A0005D085B0220040319CE
:100B3000042E5A08A8005B08A900AA01AB016008AE
:100B4000A0006108A1006208A2006308A300592068
:100B5000831203132C088316A70083122D08831613
:100B6000A80083122E088316A90083122F0883166B
:100B7000AA0027088312A000831628088312A10068
:100B8000831629088312A20083162A088312A30061
:100B90005A08A4005B08A500A601A7018A113A2003
:100BA000831203132808E0002908E1002A08E20064
:100BB0002B08E30083168A112B18FF2D831260087F
:100BC000A0006108A1006208A2006308A3005A08FF
:100BD000A0075B0803185B0FA1070030FE00031895
:100BE0007E0FA2070030FE0003187E0FA307200827
:100BF000E0002108E1002208E2002308E30083125C
:100C00005A08DC005B08DD0083162B1C292E83129A
:100C10006008A0006108A1006208A2006308A300A8
:100C20005A08A0075B0803185B0FA1070030FE00FD
:100C300003187E0FA2070030FE0003187E0FA307E3
:100C40002008E0002108E1002208E2002308E30078
:100C5000080083126008A0006108A1006208A200D9
:100C60006308A3005A08A0025B08031C5B0FA102E3
:100C70000030FE00031C7E0FA2020030FE00031CA9
:100C80007E0FA3022008E0002108E1002208E20014
:100C90002308E300080000306302031D592E98303A
:100CA0006202031D592E96306102031D592E8030B9
:100CB000600203195D2E031CA62E60088316CE0069
:100CC000831261088316CF00831262088316D00056
:100CD000831263088316D1004030CE024B30FE00F1
:100CE000031C7E0FCF024C30FE00031C7E0FD0028F
:100CF0000030FE00031C7E0FD1024E088312A000BC
:100D000083164F088312A100831650088312A20095
:100D1000831651088312A300BC30A0020230FE00EB
:100D2000031C7E0FA1020030FE00031C7E0FA202F6
:100D30000030FE00031C7E0FA3022008E4002108FF
:100D4000E5002208E6002308E700EE2E600883167F
:100D5000CE00831261088316CF00831262088316C7
:100D6000D000831263088316D1004030CE074B3089
:100D7000FE0003187E0FCF074C30FE0003187E0FD5
:100D8000D0070030FE0003187E0FD1074E088312F3
:100D9000A00083164F088312A10083165008831207
:100DA000A200831651088312A300BC30A0070230B2
:100DB000FE0003187E0FA1070030FE0003187E0F0F
:100DC000A2070030FE0003187E0FA3072008E400EE
:100DD0002108E5002208E6002308E7006408A000D7
:100DE0006508A1006608A2006708A3005608A007CE
:100DF00057080318570FA1070030D71BFF30FE001C
:100E000003187E0FA2077E0803187E0FA307200891
:100E1000E4002108E5002208E6002308E7000800B6
:100E20004B268312031360088316CE0083126108D9
:100E30008316CF00831262088316D00083126308E2
:100E40008316D10000308A11F12083120313640845
:100E50008316CE00831265088316CF0083126608BE
:100E60008316D000831267088316D10001308A11DF
:100E7000F1208312031360088316CE0083126108E9
:100E80008316CF00831262088316D0008312630892
:100E90008316D100831256088316D8008312570890
:100EA0008316D900AE30DE00DF0183128A11581B91
:100EB0005C2F031727105E2F031727145F220C30B7
:100EC00083160313CE00CF01AE30D400D50100301D
:100ED0008A1198238312031349088A116D24033061
:100EE00083120313550283164C10031D03184C1470
:100EF000CC1083128A11581F802F83164C18CC14E3
:100F00008316CC1C852F04306D2C08000B138C1C11
:100F1000B42F8C1083168C1083121211DE0A031961
:100F2000DF0AD91F962F8316A110982F8316A114BC
:100F3000003083125F02031D9F2FD0305E028316A4
:100F40002111031D03182115A115A118211DA1119F
:100F5000A11DB02F05308312DE00DF01D91759170C
:100F600083168C14831212158A150C1F5028C0305A
:100F70001F058316A000200D8312D000D00D500D48
:100F80000339D0000C1383160C1383125911591016
:100F900051088A11031DE42F01305002031DD42F84
:100FA000591559108A15072802305002031DDC2FED
:100FB000591159148A15072803305002031DE22FD6
:100FC000591559148A15072801305102031DF02FB5
:100FD000033050028A15031D072859115914072898
:100FE00002305102031DFC2F033050028A15031DED
:100FF0000728591559100728033051028A15031D77
:10100000072803305002031D0728591159105008B2
:10101000D100591C132852085302031913285208EF
:10102000D300D9145910591D4E28520854020319DF
:101030004E285208D40001305402031D2328DE013B
:10104000DF01D8134C2807305402031D4C28D81751
:1010500000305F02031D2E2802305E028316A311AA
:10106000031D0318A315003083125F02031D3A28E5
:1010700004305E0283162312031D031C2316A316DD
:10108000A319231EA312A31E4C288312581F4A28FB
:1010900058134B285817D8168312591183160C175A
:1010A0000B1C352983120608CA000B108B114A0E3F
:1010B0000F398316A000033020058312CB004A0DA0
:1010C0008316A000A00D200D0339A00003302005D9
:1010D0008312CD004B084C0203198C280530DE002A
:1010E000DF01D9134B08031D772858168A280130D1
:1010F0004B02031D7D28D8158A2802304B02031DA0
:10110000832858158A2803304B02031D8A2858115A
:10111000D81158124B08CC004E084D02031934293F
:101120000530DE00DF01D91303304E02831624138D
:101130000319241783124D084F028316A413031DAD
:10114000A4172514241BA41F2510251CFF280130DB
:1011500083124D02031DD328D81FCB28581FC52842
:10116000D60A0319D70A5708803AA0008330200214
:10117000031DBC28E730560203192D29031C2D2915
:10118000E730D6000330D7002D2983162B148A119F
:1011900090258A152D295A08EE005B08EF008A1168
:1011A00068258A152D2902304D02031D2D29D81FCF
:1011B000F728581FF128D603560A0319D7035708F2
:1011C000803AA0007C302002031DE8281930560226
:1011D00003192D2903182D291930D600FC30D7000A
:1011E0002D2983162B108A1190258A152D295A082E
:1011F000EC005B08ED008A113F258A152D2983122A
:101200004E088316A516031DA51283124D084F0222
:1012100083162513031D2517A517A51A251FA5132A
:10122000A51F2D29023083124D02031D2129D81F2D
:101230002D29581B2D2983162B148A1190258A15C8
:101240002D2901304D02031D2D29D81F2D29581B92
:101250002D2983162B108A119025831203134E0813
:10126000CF004D08CE00D8168B150B17831230080F
:10127000A0003108A1003208A2003308A3003408FE
:10128000A4003508A5003608A6003708A7003808CE
:10129000A8003908A9003A08AA003B08AB003C089E
:1012A000AC003D08AD003E08AE003F08AF00480866
:1012B00084004308C2004408FE0041088A00400E32
:1012C0008300FF0E7F0E0900831203131730A00066
:1012D000F730A1002230A2000A128A15A20B6C2955
:1012E0000A128A15A10B6A290A128A15A00B68290D
:1012F00000000000000083168113AC172C08831235
:10130000850083162C172C088312850083162C1653
:101310002C08831285008A113922083083120317A2
:10132000A2002130A3008A11B520383083120317A0
:10133000A2002230A3008A11B52083120313D60124
:10134000D7010330CC00CE01CF010530DE00DF0134
:10135000D001D101D81724308316BF00C0013F0847
:10136000DA004008DB008A11AE2483160313C100A3
:101370004108BA003A088312D50003305507D3005C
:1013800025308316BF00C0013F08CC004008CD00C7
:101390008A11DA24831603135208C1005308C200CD
:1013A0004108BA004208BB003A088312D8008316ED
:1013B0003B088312D90027308316BF00C0013F08C5
:1013C000CC004008CD008A11DA248316031352089A
:1013D000C1005308C2004108BA004208BB003A08E5
:1013E0008312DA0083163B088312DB005A08DC0004
:1013F0005B08DD008A111325031083120313550DBA
:101400008316BA000310BA0D3A08BF00C0013F08A6
:10141000CA004008CB004A08CC004B08CD008A1116
:10142000DA24831603135208C5005308C600400887
:10143000CA0002303F07C9000318CA0A4908CC0095
:101440004A08CD008A11DA24831603135208C70014
:101450005308C8004508C1004608C2004708C30039
:101460004808C4004108BA004208BB004308BC0059
:101470004408BD003A088312E00083163B0883123B
:10148000E10083163C088312E20083163D088312B4
:10149000E300D816803083169F00023083129F002D
:1014A000D2010F305205A0000F302005A100F0300E
:1014B00083161F058312210483169F007E3083123A
:1014C00092008B170B178B150B1083160C178312BA
:1014D0000C1383168C1483128C1083128A15D91C5A
:1014E000C12A03305302D5000310550D8316BA00EC
:1014F0000310BA0D3A08BF00C0013F08CA004008F7
:10150000CB004A08CC004B08CD008A11DA248316A0
:1015100003135208C5005308C6004008CA00023031
:101520003F07C9000318CA0A4908CC004A08CD0081
:101530008A11DA24831603135208C7005308C8001F
:101540004508C1004608C2004708C3004808C40057
:101550004108BA004208BB004308BC004408BD0073
:101560003A088312E00083163B088312E1008316D9
:101570003C088312E20083163D088312E300D8166C
:10158000D9108A15D81EC92A8A111027831203136D
:10159000D8128A15581DDF2A8316AC132C08831223
:1015A0008500831203134130A0000A128A15A00B94
:1015B000D72A83162C132C0883128500F12A831650
:1015C0002C172C0883128500831203134130A000CE
:1015D0000A128A15A00BEA2A8316AC172C0883126C
:1015E0008500591F622B5813591324308316DA00D3
:1015F000DB01831255088A11BC242530831603139E
:10160000CC00CD01831258088316D20083125908EA
:101610008316D3008A11F824273083160313CC00D5
:10162000CD0183125A088316D20083125B088316F9
:10163000D3008A11F824031083120313550D831667
:10164000BA000310BA0D3A08BF00C0018312600847
:101650008316C100831261088316C20083126208D8
:101660008316C300831263088316C4003F08C600B4
:101670004008C7004608CC004708CD004108D2000A
:101680004208D3008A11F824831603134008C600C9
:1016900002303F07C5000318C60A4508CC004608BB
:1016A000CD004308D2004408D3008A11F8248312E5
:1016B0000313D816831203134130A0000A128A15AF
:1016C000A00B602B83160C1F6D2A0F30831252055E
:1016D000A0000F302005A100F03083161F058312F3
:1016E000210483169F008312D20A0F30520203197D
:1016F0007B2B031C7D2BD201D101831203134130BC
:0C170000A0000A128A15A00B832B6D2A92
:02400E00383F39
:10420000E00003001C0000004000520036000000E7
:10421000F00044006B000000A0005B009A0000006A
:10422000E0008900D60000007000F80013000100D3
:10423000A000590041000100100009007C000100AD
:1042400060002900AC000100020083008000010032
:0242500000006C
:00000001FF
